:020000040000fa
:080000000002040000000000f2
:020000040000fa
:100400000fad2000807f2400000188000000000064
:100410000a00070011000700000020000000e000b3
:10042000020032000000020000000000921f0200e3
:10043000000000000040da000000fe004440a90077
:10044000000c20000000e00003003200000020004b
:10045000a00188004440a8000000060020292200d6
:10046000010020001500370062004000e0804800d5
:10047000910188009001ba0062004000e0804800cd
:10048000910188009002ba0062004000e0804800bc
:100490000002eb006028e10004003a000059eb0084
:1004a0008301e900fdff3e00040037006128e10000
:1004b000010032000082eb00050007009101880076
:1004c0001001ba000200e000e7ff3a00000005005a
:1004d000910188008002780062004000e0804800be
:1004e0003559ba008301e900080032002559ba00e5
:1004f0008301e900050032000400e000f4ff32004f
:1005000015d9ba008301e900f1ff3a0000000600a6
:100510008c02040000000000881f780002047800ac
:1005200014000700080040004f0478000000060097
:100530000000fa00881f7800000478003fb9970097
:10054000ea81570080007800c028200010000700d2
:10055000800078000000e000020035000040eb0061
:1005600000f47800010078004f0478000080fa0061
:10057000000006008001eb000200370061f0790006
:100580008301e800828f5100fcff3a000000060062
:100590006200fa00889fbe008a9fbe000004be0071
:1005a000020578008300780060f92f000f004000fa
:1005b000b000070088979f0099979f000000eb000c
:1005c000a09f9f009a4578000b80fb000000ea0086
:1005d000cf04de0050c2b30080cf550002003200cd
:1005e00009047800010037000904e9000800e00070
:1005f0000b0034001f909700080178008a007800f3
:100600008f9197000300010090979f000000e00089
:10061000930032002f98970000004400a09f9f0095
:100620000905450050c2b30080cf550004003200d8
:100630000b04e000e3ff3a002f9897008900370091
:100640000000eb00809f9f00f0979f00e0979f00c5
:10065000d0979f00c0979f00b0979f00c09f9f00ba
:1006600009003700208c200000805000000040006e
:10067000618b2000e10078004f9897000100700026
:10068000c09f9f000a05e8001a4478008800fb001c
:10069000208c20007c000700800078000000e00033
:1006a000f0ff3a00a0c2b300804f54000e003a00a1
:1006b000bf8897000180e900b08f9f00100078008c
:1006c000b09f9f000000e00005003d000000ea0030
:1006d000b09f9f004f9897000020a000c09f9f00f0
:1006e0000a05e80010003700b19f9f00090037009d
:1006f000bf989700f0ff2700808f50000400320061
:100700006a08b9000000410003004000b09f9f004c
:100710000a05e8001a01fb0003fd2f000300410059
:10072000e90f5000f2ff3600e0c2b3009a4f10000c
:10073000040032000080eb00909f9f008a04780044
:100740001c0037008a04e800a0c2b300994f1000d3
:1007500007003a00bf8897000180e900b08f9f0032
:1007600010007800909f9f008a84e80011003700f5
:100770000000eb00909f9f00090037009f989700b2
:10078000f0ff2700808f5000040032006a08b90093
:100790000000410003004000909f9f008904e80092
:1007a0001901fb0003fd2f0003004100e90f500079
:1007b000f2ff3600194478008800fb00808c20008e
:1007c000310007000000e00002003a000044780019
:1007d000010037008904e800a87f9f0080c6b300ad
:1007e000804f540004003a00994f14000a003a0068
:1007f0006640500006003700c0c6b300804f54006a
:1008000005003a00994f140003003a00654040008b
:10081000a07f9f008904e8000905e800cbfb2f00ba
:100820008f8545001901fb0060f92f000f00400083
:100830000084e8008b0178008000780008007800d0
:100840001a0007000000e00005003a008b00780065
:1008500008007800580107000000e00059ff3d0043
:100860000080eb004f05be004f04be000080fa0080
:10087000000006000200fa00f1bf9f0001087800a6
:100880000080fa0000000600040037000204e000c7
:1008900001003a00000005000000e8001041780067
:1008a000814f5100f9ff3a0000000600889fbe000a
:1008b0008a1f7800000478000102780082447800e2
:1008c00003057800e0c6b300804f5100d20032002b
:1008d00015003c006b405000804f51002400320056
:1008e0000a003c0070405000804f51000f01320060
:1008f00065404000804f51007400320050c2b30088
:10090000804f510020013a001c01370040c6b3005f
:10091000804f51001b00320065404000804f510065
:1009200019013a001700370030c7b300804f51005b
:10093000fe00320007003c0064405000804f510030
:10094000620032000040e800804f51000e013a0082
:10095000e700370050c7b300804f51005b00320002
:1009600063404000804f510007013a0057003700b4
:100970009180e900010a7800780090009171780078
:1009800007013700a8609000c0c6b30080cf5000b8
:100990000a003a009400780064805000000a780051
:1009a0001000be004f89de00cf91de000002be00c5
:1009b00002037800820378001300370010c7b300e9
:1009c00080cf500003003200a0c6b30080cf50009b
:1009d00006003a009400780068805000000a780011
:1009e0003002be002003be00070037001480e9007b
:1009f000000a78001000780000027800cfa2de0024
:100a00000503780086037800049cbe000694be00af
:100a1000a860900080c6b30080cf50000e00320066
:100a200020c6b30080cf500005003a000400fb0050
:100a3000cf80de0001017800820178000a003700d3
:100a400040c7b30080cf5000030032006640400032
:100a500080cf500006003a0004007800cf80de000e
:100a60000101780082017800009cbe000294be0063
:100a70003800be002801be00e00f5000e08f580093
:100a8000e00f5900e08f590003003d00780090000e
:100a9000d1c2b3000a003700081090000018a3006c
:100aa0000300320078009000b1c2b30004003700a8
:100ab0000008a300530032007800900001c2b30088
:100ac000017578000000e8004d003700a860900034
:100ad000c0c6b30080cf500006003a0094007800f2
:100ae00064805000000a78001002be006033b80035
:100af0001300370010c7b30080cf5000030032004e
:100b0000a0c6b30080cf500006003a0094007800e1
:100b100068805000000a78003002be002003be004a
:100b2000070037001480e900000a78001000780000
:100b300000027800050020000600200007002000c9
:100b4000049cbe000694be00a860900080c6b3005e
:100b500080cf50000e00320020c6b30080cf50007e
:100b600005003a000480fb00010020000200200084
:100b7000030020000a00370040c7b30080cf5000b8
:100b8000030032006640400080cf500006003a006b
:100b90000400780001002000020020000300200073
:100ba000009cbe000294be00081090000038a30014
:100bb000140032003800be002801be00e00f5000d3
:100bc000e08f5800e00f5900e08f59000d0032000f
:100bd00080c7b30080cf54000300320080c5b3004b
:100be00080cf540007003a007800900001c3b300a2
:100bf000017578008000e80009f578000080e800c1
:100c0000700498007800900000004500600498008f
:100c10008940780042003700a8609000c0c6b30049
:100c200080cf5000250032000a003c006440500094
:100c300080cf50002800320000c0e80080cf500074
:100c4000140032006840500080cf500022003a006b
:100c50000a00370040c7b30080cf50001e003200aa
:100c60006640400080cf50001b00320069405000b9
:100c700080cf500018003a00060037001480e900c9
:100c8000000a780010007800485c9000084878005e
:100c9000450037001480e900000a7800100278004f
:100ca00068089000cf80de000101780082017800a2
:100cb000009abe000292be003b0037001480e9009b
:100cc000000a78001001780068089000cf80de00ec
:100cd0000089be00340037001480e900000a780063
:100ce00010007800680c9000080878002e0037008b
:100cf0001180e9008008780010007800cf80de00c5
:100d00000101780082017800009cbe000294be00c0
:100d100078009000000045006004980081c7b3008f
:100d200008007800ee0007001f0037001480e9007b
:100d3000000a7800100078006004980058099000bc
:100d40000200e00002003d009d010700090037009d
:100d50008000eb00a1010700800078000000e000a7
:100d6000030032006800900000805000010037004e
:100d700058089000100c98000b0037007800900085
:100d8000027578000600370078009000800045006a
:100d90000904e00001003a0059c2b3008948780014
:100da0000000e800700498000000eb004f05780098
:100db0004f04be00000006000400fa00889fbe0039
:100dc0008a9fbe008c1f780000047800010678001e
:100dd00070089000f8009000010050008808900012
:100de000010050009808900001005000a8089000f1
:100df00001005000b808900001005000c8089000a1
:100e0000810550000002220090bf9f0000032300d4
:100e1000a0bf9f00081090000028a30018003a000f
:100e20000b00e000160034008b0478000905780000
:100e3000e28f5400020036002a0020000200370032
:100e40000900e0000b00340058009000c801900039
:100e50000a017800ee80570003000100500498005a
:100e60000000e00096003200680890000000450095
:100e7000600c98008a8454004240a900ebff3c00bb
:100e8000780190000200e0000b0034005800900050
:100e9000c80190008c007800030001005004980005
:100ea0000000e0008600320068089000f800900022
:100eb00001004000600c9800880c90000900e000e0
:100ec0001500340009057800e28f54000200360056
:100ed0002a002000020037000900e0000b00340067
:100ee00058009000c80190000a017800ec8057007b
:100ef00003000100500498000000e0007000320080
:100f00006808900000004500600c98008a84540036
:100f10004240a900ebff3c00180990000200e000ed
:100f20000b003400e800900058009000c8019000c9
:100f300003000100500498000000e000600032004f
:100f4000680890009808900001004000600c98002c
:100f5000a80c90000900e000150034000905780095
:100f6000e28f5400020036002a0020000200370001
:100f70000900e0000b00340058009000c801900008
:100f80000a017800ec80570003000100500498002b
:100f90000000e0004a0032006808900000004500b0
:100fa000600c98008a8454004240a900ebff3c008a
:100fb000380990000200e0000d003400e8009000c5
:100fc000180890008080400058009000c8019000f0
:100fd00003000100500498000000e00038003200d7
:100fe00068089000b808900001004000600c98006c
:100ff000c80c90000900e0001500340009057800d5
:10100000e28f5400020036002a0020000200370060
:101010000900e0000b00340058009000c801900067
:101020000a017800ec80570003000100500498008a
:101030000000e00022003200680890000000450037
:10104000600c98008a8454004240a900ebff3c00e9
:10105000081090000028a3001b0032000b00e000e5
:10106000190034008b04780009057800e28f5400e1
:10107000020036002a002000020037000900e000cc
:101080000b00340058009000c80190000a0178005d
:10109000ee80570003000100500498000000e000bb
:1010a000070032006808900000004500600c9800be
:1010b0008a8454004240a90003003400eaff37004c
:1010c0000080eb00010037000000eb004f067800c5
:1010d0004f05be004f04be000080fa00000006006d
:1010e000ef02b000889fbe008a9fbe008c9fbe00aa
:1010f0008e1f780000067800508a2000c0b79f003d
:1011000080c5b30080cf5000080032004289200023
:10111000c2b79f007740400080cf500003003a00e4
:1011200083002000b3b79f000a00370080c7b300d8
:1011300080cf500005003200a4002000b4b79f000b
:1011400080c5b30080cf500002003a0000012000ab
:10115000b0b79f003c04be002c05be0040c6b300e3
:1011600080cf5000030032006540400080cf500027
:101170000b003a00e00f5400e08f5c00e00f5d00d0
:10118000e08f5d0006003d006000b8006011b8000f
:1011900008045000898458000a0559008b855900bd
:1011a000e00f5400e08f5c00e00f5d00e08f5d0019
:1011b00004003a005c0890008d0120000000e0006f
:1011c0000c003200bfb0970001027800cfa2de0011
:1011d00005037800860378000800be000a01be00ff
:1011e000270207004fb2970064407800d0df9f00cd
:1011f0007d0120003fb0970000027800cfa2de0002
:1012000005037800860378000800be000a01be00ce
:1012100014020700009ebe000296be000d00e90009
:1012200061fc2f008f804000008740001e003700c7
:101230003fb1970002047800cfc4de0009057800b2
:101240008a0578000802be000a03be007fa8970046
:101250008fb097001fb19700afb197000c02070045
:10126000d0b79f00e1b79f00f2b79f0083bf9f00f8
:101270008d06e9000802be000a03be008a020700cc
:101280007faa970000005200cfb097006157780006
:101290005fb09700efb097007fb197008fb99700cc
:1012a000009ebe000296be003c00be002c01be00a7
:1012b000f0af9f0081b79f0092b79f00a3b79f0038
:1012c000e00f5000e08f5800e00f5900e08f590008
:1012d000020034000d00e000d5ff3c00bfb09700d5
:1012e000e88f500010003a000c1090000038a30066
:1012f0000d003200f78f560006003e0062fc2f0002
:101300000f0141008d00410000c3b300914f100058
:10131000050032008d06e90000c3b30063fc2f0016
:101320008f81410080f17e0078811600120e9800b6
:101330006c00900063fc2f008f8141008d80410084
:101340008cfc07001c0990005c089000800f510085
:1013500006003d0002005000000e98000c109000a6
:101360000040a100001698000f0037000000e000c8
:101370000d003d000c10900074006000f00f500054
:1013800009003a007c089000fc0090000100500029
:101390008c08900001005000020050004240a9005b
:1013a00001003400000e98004f0778004f06be0081
:1013b0004f05be004f04be00ef02b1000000060062
:1013c00080007800010037000000e8001004e00011
:1013d000fdff3a0001005000000006008001eb0014
:1013e000040037008301e80090cf100004003200b1
:1013f0000000e800828f5100faff3a000000eb0085
:1014000000000600889fbe008a9fbe008c1f7800e7
:10141000530207005a02330003866c006450e10057
:10142000240032006420e100270032006150e10016
:10143000220032006120e100210032008b85420051
:10144000eb07b1000134b800003ab80008044200cc
:1014500089844a00013ab8000030b8008880400012
:1014600009014a0004003300000040008180480068
:10147000020149008b05e900c909dd008301700004
:101480000100320013002000c814de004814dd0003
:101490004709de001200b200c808de0008847000b0
:1014a0004702070001f0a1000cf0a70001f0a00026
:1014b0003c0237006120e1003e0232000801be001c
:1014c0000200be00f7ff37006150e100fcff3a0068
:1014d000380237000001be005f0207000470a70059
:1014e00003f0a10003f8a30013003a006509b1005e
:1014f00010003200090035006928e10002003500c3
:101500000100280000000500000040008180480024
:101510008502e900fcff3a0000000600f88f420057
:10152000050035008100d1000080d3008502e8006d
:10153000fcff3a00000006008000eb000000050000
:10154000889fbe008a9fbe00010578000100e00070
:101550000400350008003c000000e00020003200dc
:101560000500370060001000e080180002003b001a
:1015700001f02c001a0037000004be006011b80012
:101580006b0920000982cf00020039000882cf00d9
:101590000441b000694252000e00320008003b00d6
:1015a00082817100610164008904d1000884d30044
:1015b0008b05e8000442e800f9ff3a000500370017
:1015c0000804440089844c008b05e9000442e900ca
:1015d000fbff3a00fa0107000af0a70001f0a000a3
:1015e0004f05be004f04be000000060003f0a2003d
:1015f000889fbe008a9fbe008c1f7800d80107001c
:10160000df0133006450e1004f0032006420e1004c
:101610005200320003826c0007003b000905d00035
:101620000306d000820f54000c065d000200390052
:101630000200320089017800030678008582550097
:1016400004003d000003fd008103fd008502ea0067
:101650008b854200840f720002003b006000100086
:10166000e08018006011b8000005eb007a28e10066
:101670000a00390006007800c75ddd00f707b200f8
:10168000878075002d003700828171000a01780083
:10169000610560008180d1000080d3008502e900ef
:1016a000f9ff3b00060440008784480002003b002d
:1016b00060041400e0841c000988a30007003200c5
:1016c0008a81710082817100610164008904d10006
:1016d0000884d3008b05e800170037000978a300c1
:1016e00013003a000b00e000130034008b05e90002
:1016f0000804440089844c000a4474000978a3005b
:101700000d003a000b00e000070034008b05e900f3
:101710000804440089844c0001003a000b002000ba
:101720000978a300f7ff32000001eb000200370048
:10173000828171000a017800a10107000cf0a70066
:1017400001f0a000970137006420e10002003a0098
:10175000838f6c00970133000801be000200be00b9
:1017600090013700f4ff2f00d00137001400200053
:10177000ce013700889fbe008a9fbe008c1f780074
:10178000770107007e01330003866c006450e1009e
:101790002e0032006420e100330032006150e1008d
:1017a0002f0032006120e1003100320085855500b4
:1017b000eb07b000090020000804200005003700f6
:1017c0000804440089844c000a00310006034300e9
:1017d00087834b000001530081815b00f8ff3300d9
:1017e0000203be000800a0000804440089844c00e5
:1017f000f6ff3900c639dd008301730001003200b5
:10180000130020008904d1000884d3000998a300a4
:10181000050032000800a7000300a0008904d100e1
:101820000884d3008b05e8008904d1000884d30024
:101830000001eb000281d2006101070001f0a1006c
:101840000cf0a70001f0a000560137006420e10071
:10185000580132000801be000200be00f7ff370049
:101860006120e100530132006000b800f3ff37004f
:101870000000200001f82700f0ff3700881f7800e3
:10188000000478005001be004000be00040040008b
:10189000858048000601490087814900009cbe0000
:1018a0000294be000400e1000588e1000690e1001a
:1018b0000798e10002003100680044001008e800c9
:1018c0004f04780000000600f4874700889fbe00a0
:1018d0008a9fbe008c9fbe008e1f78000205be004e
:1018e0000004be00d4b79f00e5b79f00f6b79f0085
:1018f00087bf9f000000eb00c0b79f00b0b79f00fc
:10190000a0b79f0090b79f0080b79f000d042000f4
:10191000bfb097004fb09700000140000000e0000a
:101920000f003d004f08de0000007100c0b79f00af
:101930009e00070001003d0012002000a1000700ea
:1019400001003d0012002000a6000700b1000700c2
:10195000b60007000f004000c8ff07002200370054
:101960004f08de0000067100ccb79f008f00070013
:1019700001003d00120020009200070001003d0020
:101980001200200097000700a20007000fb2970086
:101990009fb297002fb39700bfb39700a90007002d
:1019a0000000520081805a0002015b0083815b00cd
:1019b00080b79f0091b79f00a2b79f00b3b79f0069
:1019c0000007eb009f0007000020e10001a8e100f4
:1019d00002b0e10003b8e100010031001e00200068
:1019e0000e005600c0b79f004fb297000400e00001
:1019f0000700350010002000010020006011b80031
:101a000008047000898470000a0571008b857100dc
:101a10008d06e900beff3a000400e00003003d002f
:101a2000820007000f00400094ff07004fa89700b6
:101a30000000e00004003a000fb497009fb4970044
:101a40002fb59700bfb59700940007004f077800a7
:101a50004f06be004f05be004f04be004f01b1004f
:101a600000000600881f780018002000881f7800fa
:101a700095ff07008f87e9004f04780000000600fb
:101a8000801feb0090ff07008f87e9000000060031
:101a9000889fbe008a9fbe008c1f78006e000700e2
:101aa00007003d0073000700e00f5b00e08f5b0064
:101ab00007003d00320007000006eb00040037007d
:101ac0003400070002003d002a0007001c0020002f
:101ad00072000700e3ff07000203be000002be0021
:101ae0000c00e00001003200220007000400be00ec
:101af0000601be004f0678004f05be004f04be0031
:101b000000000600889fbe008a9fbe008c1f7800e0
:101b10005100070005003d0056000700e00f5b0084
:101b2000e08f5b0006003d0004003700190007004d
:101b300003003d006000b8006011b800100007000d
:101b400056000700ceff07000203be000002be00e1
:101b50000c00e00001003200060007000400be0097
:101b60000601be004f0678004f05be004f04be00c0
:101b7000000006006000b8006011b80000003700e7
:101b800004025000858258000603590087835900db
:101b9000000006000006eb00e00f5200e08f5a0044
:101ba000e00f5b00e08f5b0000000600018040005a
:101bb00090b79f000001eb008fb097000100e0009c
:101bc000000006000200700090b79f0001804000f6
:101bd00080b79f000001eb00ffa897000100e00024
:101be000000006000200700080b79f0001804000e6
:101bf0006faa9700cf20de0001007000f0af9f00b9
:101c000004024200250007004f18de0000027200a7
:101c100000000600e4af9f000804440089844c00e3
:101c20000a054d008b854d00000006003fb297006d
:101c3000cfb297005fb39700efb3970000fe2f007d
:101c4000000006003fb09700cfb097005fb197004b
:101c5000efb19700000006000205be000004be00c0
:101c6000e00f5000e08f5800e00f5900e08f59005e
:101c7000000006006000b8006011b80008045000c1
:101c8000898458000a0559008b8559001c002000e2
:101c9000e00f5200e08f5a00000006000800be006e
:101ca0000a01be0000000600889fbe008a9fbe0099
:101cb0008c1f78000205be000004be000006eb0089
:101cc000e00f5000e08f5800e00f5900e08f5900fe
:101cd00007003d006000b8006011b8000804500023
:101ce000898458000a0559008b8559001c00200082
:101cf000e00f5200e08f5a00e00f5b00e08f5b00c6
:101d000002003d000f0007000c00a2000800be000a
:101d10000a01be00800007000203be000002be00f0
:101d20000c00e00001003200060007000400be00c5
:101d30000601be004f0678004f05be004f04be00ee
:101d4000000006006000b8006011b80004025000f6
:101d50008582580006035900878359000000060059
:101d60000004be003c0007000003be000405be00e6
:101d70000200be0038000700844f75000000060016
:101d80000200be006450e100050036006420e1005e
:101d9000020036000968a30001003a000800be00f6
:101da0000160a0004f0678004f05be004f04be0042
:101db00000000600f0ff2f00f1ff2700f9ff3700b9
:101dc00081002000618055000b003d000b002000c9
:101dd00061fe2f000100e1001d00340082817100ce
:101de000610164008904d1000884d3000000e80088
:101df000faff3a00710020006100640003007000e7
:101e0000020060000900320061044400e0844c00dc
:101e10000988a500050032008b05e8006808e1008c
:101e200002003a008904d1000884d300f20f200098
:101e30000258e10005003d00c75ddd00f907b20072
:101e40008980750008007800000006000bf8270064
:101e50008b00780000000500c70ade00f107b20021
:101e6000f50fb20008003200e1cf4200020032005c
:101e70000170a00024000500810f700001003200f5
:101e80000408050044000500810f700002003a00bc
:101e9000140005008502e9000000400081c04800f0
:101ea000fcff3b000170a00024000500889fbe00dd
:101eb0008a9fbe00841f7800a9ff07004f007800aa
:101ec00011003300f0ff2f00838f6c0006003b00f1
:101ed000040565000a00a7000800370009f0a60005
:101ee0001000200008003700820f5400838f5c0030
:101ef000030039001000200001003e000000200017
:101f000009f0a7000000ea004f05be004f04be0024
:101f10000000e00000000600889fbe008a9fbe000f
:101f20008c9fbe000404b8000506b8008904460072
:101f300060854e000606b8000a054600e0854e00a2
:101f40000706b8008b054600040eb8008904460059
:101f50000a854e00e0854d00050eb8000a054600d2
:101f60008b854e00060eb8008b0546000416b8009f
:101f70000a0546008b854e000516b8008b05460005
:101f8000041eb8008b0546000800be000a01be0012
:101f90004f06be004f05be004f04be000000060005
:101fa0000200fa000000eb00000f780023c2bf001f
:101fb0000080fb00610060000000e00002003a00c9
:101fc00010002000000f78001e0078000080fa004a
:101fd000000006000200fa000000eb00000f78008d
:101fe00033c2bf000080fb00610060000000e00021
:101ff00002003a0010002000000f78001e00780058
:102000000080fa00000006000000fa0021e2a900aa
:102010009560a9009580a9008560a9008580a90028
:102020000080fa00000006000000fa0031e2a9007a
:1020300097c0a90097e0a90087c0a90087e0a90080
:102040000080fa00000006000200fa00000f78008d
:102050008560a9008580a9009e00780067806000e7
:10206000674060004401dd00910a20009140780043
:10207000f0c8b30000c0600002407000a9e0b700e3
:10208000000720001e0060004400de006741600081
:10209000a10a20009140780080cfb30000c060000a
:1020a00002407000aae0b7009e00780068806000df
:1020b0004300de00614060004301dd005109200063
:1020c0009140780070cfb30000c060000240700003
:1020d00095e0b700000820001e0060004700de0009
:1020e000614060004401dd0051092000914078000a
:1020f000f0ceb30000c060000240700095e0b70071
:102100000080fa00000006000200fa00000f7800cc
:1021100087c0a90087e0a9009e0078006780600062
:1021200067416000310b20009140780080cfb30000
:1021300000c0600002407000b3e0b700000720005c
:102140001e0060004400de00674060004401dd00c6
:10215000310b200091407800f0c8b30000c060004f
:1021600002407000b3e0b7009e0078006880600015
:102170004300de00614060004601dd00710920007f
:1021800091407800f0cbb30000c0600002407000c6
:1021900097e0b700000820001e0060004700de0046
:1021a000c700dd0097c0bf000074a10001407000af
:1021b00097e0b7000080fa00000006000000fa0077
:1021c00022c2bf000080fb00610060000000fb0035
:1021d0000080fa00000006000000fa0032c2bf00d2
:1021e0000080fb00610060000000fb000080fa003e
:1021f000000006000c00fa00000f7800110798009c
:10220000220798000000eb00300798001e009000a5
:10221000400798001e00e00029003200e7ff070099
:102220000004e0000b003a00be0090002e00900079
:10223000808f5000040031003e0090000000e80054
:1022400030079800f5ff37001e007800500798000f
:102250001d0037000000eb003007980020c2bf00cf
:102260000080fb000000d1000080fb0063006000e4
:10227000e30f500008003a000e80e800900078005c
:102280000101780033118000030978008180e800a3
:102290000108780008003700e80147009300780043
:1022a0003011800000417800010078000248780079
:1022b0008100e800810978001e0fe900d5ff370092
:1022c0001e007800500798005e0090000080fa0021
:1022d000000006000c00fa00000f780011079800bb
:1022e000220798000000eb00300798001e009000c5
:1022f000400798001e00e00029003200b6ff0700ea
:102300000004e0000b003a00be0090002e00900098
:10231000808f5000040031003e0090000000e80073
:1023200030079800f5ff37001e007800500798002e
:102330001d0037000000eb003007980030c2bf00de
:102340000080fb000000d1000080fb006300600003
:10235000e30f500008003a000e80e800900078007b
:1023600001017800b3118000030978008180e80042
:102370000108780008003700e80147009300780062
:10238000b011800000417800010078000248780018
:102390008100e800810978001e0fe900d5ff3700b1
:1023a0001e007800500798005e0090000080fa0040
:1023b000000006000600fa00000f780011079800e0
:1023c000220798002e009000401188001e0078001f
:1023d000001188001e009000101188000080fa0093
:1023e000000006000600fa00000f780011079800b0
:1023f000220798002e009000c01188001e0078006f
:10240000801188001e009000901188000080fa0062
:10241000000006000400fa00000f78001e0078009b
:102420001007980023c2bf000080fb000000d1000d
:102430000080fb00610060000000e000f9ff3a004e
:1024400020c2bf000080fb000000d1000080fb0024
:1024500063006000e30f50000f003a001e00780098
:102460001000e0001e0032001e007800100078000e
:10247000201188001e8fe80023c2bf000080fb00ef
:102480000000d1000080fb00610060000000e0005f
:10249000f9ff3a00f1ff37001e0090001004e00041
:1024a0000f0032000e81e8001200780080007800f2
:1024b0009100fb00211188000000e800000978006d
:1024c00023c2bf000080fb000000d1000080fb00a1
:1024d000610060000000e000f9ff3a00eeff370005
:1024e0000080fa00000006000400fa00000f7800e7
:1024f0001e0078001007980033c2bf000080fb0068
:102500000000d1000080fb00610060000000e000de
:10251000f9ff3a0030c2bf000080fb000000d1008c
:102520000080fb0063006000e30f50000f003a00e2
:102530001e0078001000e0001e0032001e0078002f
:1025400010007800a01188001e8fe80033c2bf0081
:102550000080fb000000d1000080fb0061006000f3
:102560000000e000f9ff3a00f1ff37001e00900084
:102570001004e0000f0032000e81e8001200780025
:10258000800078009100fb00a11188000000e800a5
:102590000009780033c2bf000080fb000000d100ba
:1025a0000080fb00610060000000e000f9ff3a00dd
:1025b000eeff37000080fa00000006000200fa007b
:1025c00020c2bf000080fb000000d1000080fb00a3
:1025d00063006000e30f500003003a0030118000f8
:1025e000000f78000400370030118000f10f200048
:1025f00001006000000f78001e0078000080fa00e3
:10260000000006000200fa0030c2bf000080fb009c
:102610000000d1000080fb0063006000e30f500069
:1026200003003a00b0118000000f7800040037006a
:10263000b0118000f10f200001006000000f780051
:102640001e0078000080fa00000006000200fa0078
:10265000000f780023c2bf000080fb000000d10003
:102660000080fb00610060000000e000f9ff3a001c
:1026700020c2bf000080fb000000d1000080fb00f2
:1026800063006000e30f500003003a001e00780072
:102690002011880003003700f00f20001e006000aa
:1026a000201188000080fa00000006000200fa00f5
:1026b000000f780033c2bf000080fb000000d10093
:1026c0000080fb00610060000000e000f9ff3a00bc
:1026d00030c2bf000080fb000000d1000080fb0082
:1026e00063006000e30f500003003a001e00780012
:1026f000a011880003003700f00f20001e006000ca
:0c270000a01188000080fa000000060014
:020000040000fa
:0200000401f009
:04000000ffff0000fe
:020000040000fa
:0200000401f009
:04000400ffff0000fa
:020000040000fa
:0200000401f009
:04000c00faff0000f7
:020000040000fa
:0200000401f009
:040010007eff00006f
:020000040000fa
:0200000401f009
:040014007fff00006a
:020000040000fa
:0200000401f009
:04001800ffff0000e6
:020000040000fa
:1000080004250000ae200000b8200000c220000037
:10001800cc20000004250000042500000425000071
:100028000425000004250000042500000425000024
:100038000425000004250000042500000425000014
:100048000425000004250000042500004c240000bd
:1000580004250000042500000425000004250000f4
:1000680004250000361d00000425000004250000ba
:1000780004250000042500000425000004250000d4
:1000880004250000042500000425000004250000c4
:1000980004250000042500008a240000042500002f
:1000a80004250000042500000425000004250000a4
:1000b8000425000004250000042500000425000094
:1000c8000425000004250000042500000425000084
:1000d8000425000004250000042500000425000074
:1000e8000425000004250000042500000425000064
:1000f8000425000004250000042500000425000054
:100108000425000004250000042500000425000043
:100118000425000004250000042500000425000033
:100128000425000004250000042500000425000023
:100138000425000004250000042500000425000013
:100148000425000004250000042500000425000003
:1001580004250000042500000425000004250000f3
:1001680004250000042500000425000004250000e3
:1001780004250000042500000425000004250000d3
:1001880004250000042500000425000004250000c3
:1001980004250000042500000425000004250000b3
:1001a80004250000042500000425000004250000a3
:1001b8000425000004250000042500000425000093
:1001c8000425000004250000042500000425000083
:1001d8000425000004250000042500000425000073
:1001e8000425000004250000042500000425000063
:0801f8000425000004250000ad
:020000040000fa
:1002080004250000ae200000b8200000c220000035
:10021800cc2000000425000004250000042500006f
:100228000425000004250000042500000425000022
:100238000425000004250000042500000425000012
:100248000425000004250000042500004c240000bb
:1002580004250000042500000425000004250000f2
:1002680004250000361d00000425000004250000b8
:1002780004250000042500000425000004250000d2
:1002880004250000042500000425000004250000c2
:1002980004250000042500008a240000042500002d
:1002a80004250000042500000425000004250000a2
:1002b8000425000004250000042500000425000092
:1002c8000425000004250000042500000425000082
:1002d8000425000004250000042500000425000072
:1002e8000425000004250000042500000425000062
:1002f8000425000004250000042500000425000052
:100308000425000004250000042500000425000041
:100318000425000004250000042500000425000031
:100328000425000004250000042500000425000021
:100338000425000004250000042500000425000011
:100348000425000004250000042500000425000001
:1003580004250000042500000425000004250000f1
:1003680004250000042500000425000004250000e1
:1003780004250000042500000425000004250000d1
:1003880004250000042500000425000004250000c1
:1003980004250000042500000425000004250000b1
:1003a80004250000042500000425000004250000a1
:1003b8000425000004250000042500000425000091
:1003c8000425000004250000042500000425000081
:1003d8000425000004250000042500000425000071
:1003e8000425000004250000042500000425000061
:0803f8000425000004250000ab
:020000040000fa
:10270c002530000032580000202500003032000037
:10271c005820000025300000325800002025000011
:10272c0030320000582000002530000032580000e4
:10273c002025000030320000582000002025000029
:10274c0030320000582000002530000032580000c4
:10275c0020250000303200005820000025300000f9
:10276c0032580000202500003032000058200000b4
:10277c0025300000325800002020000025300000d9
:10278c003258000020250000303200005820000094
:10279c0025300000325800002025000030320000a7
:1027ac005820000025300000325800002025000081
:1027bc0030320000582000000a0d0000000000001c
:020000040000fa
:1027cc000600fa00004f78001e4078004047980041
:1027dc004e4090000004e00020003200803e2000bb
:1027ec00100798001e0090000000e000140032005a
:1027fc00cbc2bf000080fb000000d1000080fb00ba
:10280c00610060000000e00005003a00cb22a80047
:10281c0000f42100010020006a08070004003700c2
:10282c00cb22a90000f4210001002000650807005c
:10283c001e0090000000e90010079800e9ff370027
:10284c0000902000d10320005e0807004e4090004d
:10285c000040e90040479800ddff37000080fa0097
:10286c00000006000400fa0000d420003100200013
:10287c00008fbe001e00be00e00f5000e08f58001d
:10288c0015003200cbc2bf000080fb000000d1005d
:10289c000080fb00610060000000e00005003a00d1
:1028ac00cb22a80000f421000100200045080700fd
:1028bc0004003700cb22a90000f421000100200005
:1028cc00400807000080eb008080eb001e0f4000ea
:1028dc005e974800e7ff37000080fa000000060012
:1028ec000000fa00cbc2bf000080fa000000060016
:1028fc000600fa00000f78000000eb00200798009b
:10290c002e0090009e0f50000e0031000000eb00d6
:10291c00100798009e00900070382100808f5000a6
:10292c0004003e001e0090000000e8001007980014
:10293c00f8ff37002e0090000000e80020079800f8
:10294c00efff37000080fa00000006000600fa00d6
:10295c00000f78000000eb00200798002e0090007c
:10296c009e0f50000d0031000000eb001007980086
:10297c001e009000e40f500004003e001e0090006a
:10298c000000e80010079800f9ff37002e009000b7
:10299c000000e80020079800f0ff37000080fa00e4
:1029ac00000006000400fa000000eb0057070700c7
:1029bc006044880060448000cf80de00ddfa0700b0
:1029cc00008fbe008c08e20005003d0002002000d4
:1029dc00037824001e00be0002fb0700008fbe001f
:1029ec0092282d00e3b523001e00be0082fa0700da
:1029fc0082612200b3fc2300f9fa070070448800be
:102a0c0081448800020020000313240070448000dd
:102a1c008144800050fb07000000e00002003400fd
:102a2c00caa2a9000a003700a29929009312240017
:102a3c00704480008144800049fb07000000e000e6
:102a4c0002003d00caa2a80001003700caa2a800db
:102a5c000080fa00000006000a00fa00004f78001f
:102a6c0011479800224798003347980064004700ac
:102a7c00400798004e009000be409000014878003e
:102a8c004e0090000000e800ae4090000148780035
:102a9c004e0090000080e8009e40900001487800b5
:102aac004e009000630040001e4878002e009000fd
:102abc00be0090000080fa00000006000400fa003e
:102acc00008fbe00b2fd2000930424001e00be0047
:102adc0025fb0700020020004333240046fa0700c0
:102aec000080fa00000006000400fa00008fbe000f
:102afc00b2fd2000930424001e00be003efa070025
:102b0c00020020004333240017fb07000080fa006a
:102b1c00000006001000fa00008fbe00220798008b
:102b2c003307980044079800550798002e01900031
:102b3c00be0190001e00be0007fb07000000e00075
:102b4c001b0034004e019000de0190001e00be0000
:102b5c0003fb07000000e00004003d001e00be0067
:102b6c0060079800710798002b0037002e01900029
:102b7c00be0190004e009000de009000f6fa0700b7
:102b8c000000e000050034004e009000de009000d4
:102b9c0060079800710798001f0037002e00900006
:102bac00be00900060079800710798001a0037006b
:102bbc004e019000de0190001e00be00e6fa0700f8
:102bcc000000e000040034001e00be006007980006
:102bdc0071079800100037002e019000be01900084
:102bec004e009000de009000ddfa07000000e000cf
:102bfc0005003d004e009000de009000600798003c
:102c0c0071079800040037002e009000be00900061
:102c1c0060079800710798006e009000fe0090000d
:102c2c000080fa00000006000800fa00000f78008f
:102c3c0011079800220798001e0090009e0f1000ac
:102c4c00100036002e0090009e0f10000300310083
:102c5c001e0078003007980019003700ae00900075
:102c6c001e009000808f5000030036002e00900054
:102c7c0030079800120037001e00900030079800b3
:102c8c000f0037002e0090009e0f1000030036003e
:102c9c001e0078003007980009003700ae00900045
:102cac001e009000808f5000030031002e00900019
:102cbc0030079800020037001e0090003007980083
:102ccc003e0090000080fa00000006000c00fa00a4
:102cdc00000f78001107980022079800330798001e
:102cec00440798001e0090009e0f10004500310014
:102cfc002e0090009e0f1000420031003e0090000c
:102d0c009e0f10003f0031004e0090009e0f1000ef
:102d1c003c003100ce0090003e009000808f5000af
:102d2c000e003600ce0090002e009000808f5000d8
:102d3c000a003600ce0090001e009000808f5000dc
:102d4c00060036003e019000ae0090001e00900080
:102d5c00b5ff0700500798003a013700be009000fd
:102d6c004e009000808f50000e003600be00900088
:102d7c002e009000808f50000a003600be0090009c
:102d8c001e009000808f5000060036004e0190000f
:102d9c00ae0090001e009000a3ff070050079800a3
:102dac0028013700ae0090004e009000808f50003c
:102dbc000e003600ae0090003e009000808f500058
:102dcc000a003600ae0090001e009000808f50006c
:102ddc00060036004e019000be0090001e009000d0
:102dec0091ff070050079800160137004e01900024
:102dfc00be0090002e0090008bff0700500798003b
:102e0c00100137001e0090009e0f5000450031004d
:102e1c009e0090002e009000808f500041003100e9
:102e2c009e0090003e009000808f50003d003100cd
:102e3c009e0090004e009000808f500039003100b1
:102e4c00ce0090003e009000808f50000d003600a8
:102e5c00ce0090002e009000808f500009003600ac
:102e6c004e0090009e0f5000060036003e01900070
:102e7c00ae0090001e0078006bff07005007980012
:102e8c00f0003700be0090004e009000808f500084
:102e9c000d003600be0090002e009000808f500078
:102eac00090036003e0090009e0f500006003600d0
:102ebc004e019000ae0090001e0078005aff0700f3
:102ecc0050079800df003700ae0090004e009000d5
:102edc00808f50000d003600ae0090003e00900038
:102eec00808f5000090036002e0090009e0f50007d
:102efc00060036004e019000be0090001e007800c7
:102f0c0049ff070050079800ce0037004e01900093
:102f1c00be0090002e00900043ff07005007980061
:102f2c00c80037002e0090009e0f50004500310065
:102f3c00ae0090001e009000808f500041003100c8
:102f4c00ae0090003e009000808f50003d0031009c
:102f5c00ae0090004e009000808f50003900310080
:102f6c00ce0090003e009000808f50000d00360087
:102f7c00ce0090001e009000808f5000090036009b
:102f8c004e0090009e0f5000060036003e0190004f
:102f9c009e0090001e00780023ff07005007980049
:102fac00a8003700be0090004e009000808f5000ab
:102fbc000d003600be0090001e009000808f500067
:102fcc00090036003e0090009e0f500006003600af
:102fdc004e0190009e0090001e00780012ff07002a
:102fec0050079800970037009e0090004e0090000c
:102ffc00808f50000d0036009e0090003e00900027
:10300c00808f5000090036001e0090009e0f50006b
:10301c00060036004e019000be0090001e007800a5
:10302c0001ff070050079800860037004e01900002
:10303c00be0090001e009000fbfe07005007980099
:10304c00800037003e0090009e0f5000450031007c
:10305c00be0090001e009000808f50004100310097
:10306c00be0090002e009000808f50003d0031007b
:10307c00be0090004e009000808f5000390031004f
:10308c00ce0090002e009000808f50000d00360076
:10309c00ce0090001e009000808f5000090036007a
:1030ac004e0090009e0f5000060036002e0190003e
:1030bc009e0090001e007800dbfe07005007980071
:1030cc0060003700ae0090004e009000808f5000e2
:1030dc000d003600ae0090001e009000808f500056
:1030ec00090036002e0090009e0f5000060036009e
:1030fc004e0190009e0090001e007800cafe070052
:10310c00500798004f0037009e0090004e00900032
:10311c00808f50000d0036009e0090002e00900015
:10312c00808f5000090036001e0090009e0f50004a
:10313c00060036004e019000ae0090001e00780094
:10314c00b9fe0700500798003e0037004e01900072
:10315c00ae0090001e009000b3fe070050079800d0
:10316c0038003700be0090002e009000808f500079
:10317c000d003600be0090001e009000808f5000a5
:10318c00090036003e0090009e0f500006003600ed
:10319c002e0190009e0090001e007800a2fe0700f9
:1031ac005007980027003700ae0090003e009000ba
:1031bc00808f50000d003600ae0090001e00900075
:1031cc00808f5000090036002e0090009e0f50009a
:1031dc00060036003e0190009e0090001e00780014
:1031ec0091fe070050079800160037009e009000d3
:1031fc003e009000808f50000d0036009e00900025
:10320c002e009000808f5000090036001e009000a8
:10321c009e0f5000060036003e019000ae0090005c
:10322c001e00780080fe070050079800050037004c
:10323c003e019000ae0090001e0090007afe070048
:10324c00500798005e0090000080fa000000060015
:10325c000800fa00008fbe006011b8001e00be000e
:10326c003ff907000000e00005003d001e00be0015
:10327c0001f0a200200798003107980003003700e6
:10328c001e00be0020079800310798002e00900009
:10329c00be0090000080fa00000006000600fa0054
:1032ac00000f78001e007800100798000e80e800d0
:1032bc00200798002e0090001080fb000080fa0080
:1032cc00000006000600fa00000f78001e007800cf
:1032dc00100798000e80e800200798002e00900040
:1032ec000000e8001080fb000080fa0000000600df
:020000040000fa
:1032fc000000fa000000000006c2bf000080fb00c6
:10330c00610060000000e000fbff3a0006c2bf0055
:10331c000080fb004200de000080fb0061006000ca
:10332c000000e000f4ff3a0006c2bf000080fb0082
:10333c004300de000080fb00610060000000e00044
:10334c00edff3a0006c2bf000080fb004400de0027
:10335c000080fb00610060000000e000e6ff3a0026
:10336c0009c2bf000080fb004600de000080fb00ad
:10337c00610060000000e000dfff3a000080fa000e
:10338c00000006000000fa0007e2a90007a2a9004d
:10339c000782a8000762a9000742a9000722a8001b
:1033ac000702a90006e2a90006c2a90006a2a9000c
:1033bc000682a9000662a9000642a9000622a900fd
:1033cc000602a900f005200020108800c10a200088
:1033dc0091407800f0c8b30000c0600001c5b30094
:1033ec0001407000ace0b70008c2a9009600a9002b
:1033fc0007e2a80000a82100610020007105070069
:10340c00100020000080fa00000006000000fa0006
:10341c0007e2a9008620a9008600a9009600a90051
:10342c00d8ff07000600070000fa2000010020006a
:10343c0064050700100020000080fa000000060060
:10344c000000fa008620a9009620a8000032200077
:10345c00010020005b050700100020000080fa002e
:10346c00000006000000fa008620a9009620a900a2
:10347c00100020000080fa00000006000600fa0090
:10348c000000000016c2bf000080fb00610060005d
:10349c000000e000fbff3a0016c2bf000080fb00fa
:1034ac004200de000080fb00610060000000e000d4
:1034bc00f4ff3a0016c2bf000080fb004300de00a0
:1034cc000080fb00610060000000e000edff3a00ae
:1034dc0016c2bf000080fb004400de000080fb0031
:1034ec00610060000000e000e6ff3a0016c2bf0079
:1034fc000080fb000000d1000080fb006100600038
:10350c000000e000dfff3a0010c0b30092e8b70003
:10351c0008c2bf000080fb004400de000080fb00fe
:10352c00610060000000e000150032000602a800f7
:10353c000071220001002000008fbe001e00be00a2
:10354c00e00f5000e08f58000a0032009248e20071
:10355c0003003a0010002000200798000a003700f2
:10356c000080eb008080eb001e0f40005e9748004f
:10357c00f2ff37008000eb002107980002003700b3
:10358c000000eb00200798002e0090000080fa004d
:10359c00000006000600fa0060c0b30092e8b70015
:1035ac0008c2bf000080fb004300de000080fb006f
:1035bc00610060000000e000150032000622a80047
:1035cc000071220001002000008fbe001e00be0012
:1035dc00e00f5000e08f58000a0032009248e200e1
:1035ec0003003a0010002000200798000a00370062
:1035fc000080eb008080eb001e0f40005e974800bf
:10360c00f2ff37008000eb00210798000200370022
:10361c000000eb00200798002e0090000080fa00bc
:10362c00000006000200fa0030c0b30092e8b700b8
:10363c0006c2bf000080fb00610060000000e000db
:10364c001c003a0006c2bf000080fb004200de00f6
:10365c000080fb00610060000000e00015003a00f3
:10366c0006c2bf000080fb004300de000080fb00b0
:10367c00610060000000e0000e003a0006c2bf00ce
:10368c000080fb004400de000080fb006100600055
:10369c000000e00007003a0006c2bf000080fb00fb
:1036ac000000d1000080fb00610060000000e00021
:1036bc00030032000000eb00000f78000900370017
:1036cc0006a2a9000682a8009248e20003003a0074
:1036dc0010002000000f7800020037000000eb0003
:1036ec00000f78001e0078000080fa000000060031
:1036fc000600fa0030c0b30092e8b70006c2bf0063
:10370c000080fb00610060000000e0001c003a003b
:10371c0006c2bf000080fb004200de000080fb0000
:10372c00610060000000e00015003a0006c2bf0016
:10373c000080fb004300de000080fb0061006000a5
:10374c000000e0000e003a0006c2bf000080fb0043
:10375c004400de000080fb00610060000000e0001f
:10376c0007003a0006c2bf000080fb000000d10039
:10377c000080fb00610060000000e00003003200ec
:10378c000000eb00200798001500370006a2a800e7
:10379c000682a8000071220001002000008fbe00ec
:1037ac001e00be00e00f5000e08f58000a003200ef
:1037bc009248e20003003a00110020002107980013
:1037cc00070037000080eb008080eb001e0f4000ec
:1037dc005e974800f2ff37008000eb00210798004d
:1037ec002e0090000080fa00000006000a00fa008b
:1037fc00000f7800007122000100200010079800d3
:10380c00210798000040eb006047980040c0b300cf
:10381c0092e8b70000712200010020001007980008
:10382c00210798001e009000ae009000e00f5000a1
:10383c00e08f58002b00320006c2bf000080fb0056
:10384c00610060000000e0001f003a0006c2bf00eb
:10385c000080fb004200de000080fb006100600085
:10386c000000e00018003a0006c2bf000080fb0018
:10387c004300de000080fb00610060000000e000ff
:10388c0011003a0006c2bf000080fb004400de00bd
:10389c000080fb00610060000000e0000a003a00bc
:1038ac0009c2bf000080fb004600de000080fb0068
:1038bc00610060000000e00003003a0010c0b3009b
:1038cc0060479800070037001e009000ae00900083
:1038dc0061005000e0805800100798002107980004
:1038ec00d0ff37006e4090000004e00003003a0067
:1038fc000000eb00400798001b0037000662a80090
:10390c00006a280011002000100798002107980079
:10391c001e009000ae009000e00f5000e08f5800a9
:10392c000f0032009248e20006003a009e00780038
:10393c00001080008048780010002000400798009c
:10394c00090037001e009000ae009000610050008e
:10395c00e08058001007980021079800ecff370012
:10396c000000eb00400798004e0090000080fa0029
:10397c00000006000600fa0050c0b30092e8b70041
:10398c000642a8000071220001002000008fbe003a
:10399c001e00be00e00f5000e08f58000a003200fd
:1039ac009248e20003003a00100020002007980023
:1039bc00070037000080eb008080eb001e0f4000fa
:1039cc005e974800f2ff37008000eb00210798005b
:1039dc002e0090000080fa00000006000800fa009b
:1039ec00004f780020c0b30092e8b7001e00fb0027
:1039fc00101088000602a8000071220001002000af
:103a0c0010079800210798001e009000ae0090004f
:103a1c00e00f5000e08f58000c0032009248e2009a
:103a2c0003003a001000200030079800090037000e
:103a3c001e009000ae00900061005000e080580025
:103a4c001007980021079800efff37000000eb00eb
:103a5c00300798003e0090000080fa00000006003d
:103a6c00801f78000000fa008620a9000040eb00bf
:103a7c0092e8b7000080fa004f0078000040060082
:020000040000fa
:103a8c000400fa00004f7800114798000040eb004a
:103a9c00204798002e4090000004e0002b003a00d4
:103aac0010c0b3002047980074fe070080407800d7
:103abc002e40900001406000204798001e40780086
:103acc00c6ff0700804078002e4090000140600047
:103adc00204798001e409000c0ff070080407800ef
:103aec002e4090000140600020479800a9fe07007e
:103afc00804078002e4090000140600020479800e4
:103b0c001e40e800b5ff0700804078002e40900072
:103b1c0001406000204798006300470033ff070016
:103b2c00804078002e4090000140600020479800b3
:103b3c00effe07008fff07002e4090000004e0000e
:103b4c0002003a0031fe0700d2ff37003e409000e1
:103b5c000000fb000080fa00000006000800fa00dc
:103b6c00004f78001107980042479800534798007f
:103b7c000040eb006047980010c0b300604798000d
:103b8c003efe0700804078006e40900001406000cf
:103b9c00604798001e40780090ff07008040780036
:103bac006e40900001406000604798004e409000cd
:103bbc008aff0700804078006e4090000140600052
:103bcc006047980073fe0700804078006e409000bc
:103bdc0001406000604798001e40e8007fff07002e
:103bec00804078006e409000014060006047980073
:103bfc005e4090000004e000210032001e009000a6
:103c0c00fafe0700804078006e4090000140600092
:103c1c00604798001e0090000000e8001007980014
:103c2c005e4090000040e900504798005e409000d4
:103c3c000004e00005003a00adfe0700ee409000e5
:103c4c0000c06000604798000400370075fe070054
:103c5c00ee40900000c0600060479800000000003b
:103c6c0006c2bf000080fb004400de000080fb00a9
:103c7c0061006000e10f5000f9ff3200dcff3700fb
:103c8c003cff07006e4090000000fb000080fa0033
:103c9c00000006000400fa00004f7800114798005d
:103cac00224798000040eb00304798003e409000bf
:103cbc000004e00023003a0010c0b3003047980025
:103ccc00eefd0700804078003e409000014060000f
:103cdc00304798001e40780040ff07008040780075
:103cec003e40900001406000304798001e4090001c
:103cfc003aff0700804078003e4090000140600091
:103d0c00304798002e40900034ff07008040780028
:103d1c003e409000014060003047980015ff0700be
:103d2c00804078003e409000014060003047980091
:103d3c003e4090000004e00002003a00b3fd070092
:103d4c00daff37003e4090000000fb000080fa00d4
:103d5c00000006000400fa00000f78000040eb00a1
:103d6c00204798000040eb00304798002e40900010
:103d7c000004e0002f003a0010c0b3002047980068
:103d8c00befd0700804078002e409000014060008e
:103d9c002047980000c1b30010ff07008040780056
:103dac002e409000014060002047980010c0b300e6
:103dbc000aff0700804078002e4090000140600010
:103dcc0020479800f3fd0700804078002e409000bb
:103ddc00014060002047980010c1b300fffe0700af
:103dec00804078002e4090000140600020479800f1
:103dfc00630047007dfe0700804078002e40900055
:103e0c00014060002047980039fe07008040780090
:103e1c002e4090000140600020479800d5fe07001e
:103e2c00804078002e4090000140600020479800b0
:103e3c00ceff37003e4090000000fb000080fa00ef
:103e4c00000006000400fa00000f780021479800db
:103e5c000040eb00304798003e4090000004e0002a
:103e6c001f003a0010c0b3003047980083fd0700d4
:103e7c00804078003e409000014060003047980040
:103e8c0000c1b300d5fe0700804078003e40900092
:103e9c0001406000304798000040eb00cffe070067
:103eac00804078003e409000014060003047980010
:103ebc0050c0b300c9fe0700804078003e4090001f
:103ecc000140600030479800aafe0700804078004f
:103edc003e4090000140600030479800deff370004
:103eec000080fa00000006000000fa0025fd070023
:103efc000080fa00000006000000fa0050fd0700e8
:103f0c000080fa00000006000000fa0055fd0700d2
:083f1c000080fa00000006001d
:020000040000fa
:103f24009001fa00a000070000482800e1012000e9
:103f3400a602070095020700120107002d010700e1
:103f4400ebff0700eeff070000482800e101200016
:103f54009e0207000040eb00a2fe0700ca22a80050
:103f6400caa2a90030c0b30017fa0700002021003c
:103f7400a107200095020700d5c2bf000080fb0006
:103f84004300de000080fb00610060000000e000f0
:103f940001003a000502070000000000810c200027
:103fa4008e80400043c1b30002c6b30000c1b30019
:103fb400ecfe0700800c20000e0040002050900012
:103fc4000080fb00801f7800800c20000e00400061
:103fd400105090000080fb00801f7800800c2000af
:103fe4000e004000005090000080fb00801f78000d
:103ff400800c20000e004000704890000080fb0000
:10400400801f7800800c20000e0040006048900063
:104014000080fb00801f7800800c20000e00400010
:10402400504890000080fb00801f7800800c200026
:104034000e004000404890000080fb00801f780084
:10404400800c20000e004000304890000080fb00ef
:10405400801f7800800c20000e0040002048900053
:104064000080fb00801f7800800c20000e004000c0
:10407400104890000080fb00801f7800800c200016
:104084000e004000004890000080fb00801f780074
:10409400800c20000e004000704090000080fb0067
:1040a400801f7800800c20000e00400060409000cb
:1040b4000080fb00801f7800800c20000e00400070
:1040c400504090000080fb00801f7800800c20008e
:1040d4000e004000404090000080fb00801f7800ec
:1040e400800c20000e004000304090000080fb0057
:1040f400801f7800800c20000e00400020409000bb
:104104000080fb00801f7800800c20000e0040001f
:10411400104090000080fb00801f78006038290068
:10412400801f78000e00780000f10700a0fd2f002a
:1041340080874700a6f707000004e000fdff3a006f
:104144000e007800e7f80700a1f707000004e0007c
:10415400fdff3a0091ff37000000fa008020a9001b
:104164000000fe000080fa00004006000000fa0093
:104174008060a9000000fe000080fa0000400600f4
:104184000000fa008040a9000000fe000080fa0050
:10419400004006000000fa008080a9000000fe0034
:0841a4000080fa000040060053
:020000040000fa
:1041ac000400fa00417420009140780000ceb30066
:1041bc0000c060003040b30044e7b70044c7bf0004
:1041cc00f043b20044e7b700e0012000303a880029
:1041dc000000eb00403a880040a7a9003200200004
:1041ec0081072000a0092000337420008149780049
:1041fc008049780082497800030f78001200200073
:10420c00610420007005200023742000814978008f
:10421c0080497800824978001307980043c7bf0093
:10422c000080fb004400de000080fb0067006000a3
:10423c00e30f5000f9ff3a000000000042c7bf0036
:10424c000080fb004500de000080fb006100600088
:10425c00e10f5000f9ff3a000080fa000000060060
:10426c000000fa000000eb00200888008460a90020
:10427c00510a200091407800f0c8b30000c06000e3
:10428c0001c5b30001407000a5e0b7000000eb00d1
:10429c000008880000c42900100888000080fa007b
:1042ac00000006000000fa009460a80005e1a800d8
:1042bc000080fa00000006000000fa009460a900db
:1042cc0005e1a9000080fa00000006000000fa00d9
:1042dc000000eb00900888008500a900810a2000ee
:1042ec009140780080cfb30000c060005040b30014
:1042fc00a8e0b7000000eb00500888000080fa002e
:10430c00000006000000fa009500a80013e1a800c8
:10431c000080fa00000006000000fa009500a900d9
:10432c0013e1a9000080fa00000006000400fa0066
:10433c00008fbe0002002400c33124001e00be000a
:10434c002df4070060f40700d00888000003280053
:10435c00f0088800110b200091407800f0c8b300e1
:10436c0000c060000044a000b1e0b7008760a90065
:0c437c009760a8000080fa000000060016
:020000040000fa
:104388000600fa001ef7070070052000000f7800ed
:10439800f0fd2f002af7070080c02c0010079800b6
:1043a800d0752900200798001e017800ae00900003
:1043b8001e009000fdf707000000eb000042880097
:1043c8000000eb00104288000080fa0000000600a0
:1043d8000000fa00eaff07000080fa00000006006b
:1043e8000000fa00020007000080fa000000060042
:1043f8000600fa000af7070070052000000f780091
:10440800f0fd2f003ef7070080602c001007980091
:10441800d0752900200798001e017800ae00900092
:104428001e009000edf707000000eb003044880004
:104438000000eb00404488000080fa0000000600fd
:104448000c00fa0070052000000f780070052000ad
:1044580010079800f0fd2f00f9f6070080c02c0027
:1044680020079800910a200091407800f0c8b30016
:1044780000c0600001c2b30001407000a9e0b700ad
:10448800a10a20009140780080cfb30000c06000ee
:104498000014a000aae0b70080802c002007980034
:1044a800005028003007980090fb2f0014f70700f1
:1044b800310b20009140780080cfb30000c060002d
:1044c8003040b300b3e0b700310b200091407800d2
:1044d800f0c8b30000c0600001c3b3000140700021
:1044e800b3e0b70080602c0040079800d075290021
:1044f800500798001e017800be0090002e00900022
:10450800aaf707001e019000de0090004e00900000
:0c451800b2f707000080fa000000060067
:020000040000fa
:104524009208000002000000000000008c08000057
:10453400060000000200000000000000000000006f
:104544000008000046000000020000000000000017
:104554000000000000000000000000000000000057
:104564000000000000000000000000000000000047
:104574000000000000000000000000000000000037
:104584000000000000000000000000000000000027
:104594000000000000000000000000000000000017
:1045a40000000000000000000000000046080000b9
:1045b40046000000020000000000000000000000af
:1045c40000000000000000000000000000000000e7
:1045d40000000000000000000000000000000000d7
:1045e40000000000000000000000000000000000c7
:1045f40000000000000000000000000000000000b7
:1046040000000000000000000000000000000000a6
:104614000000000000000000b608000012000000c6
:104624000200000001000200000400000800100065
:1046340000000000202b2d0023300000c8080000db
:104644000800000002000000686a6c00747a4c00e4
:104654000000000094080000220000000200000096
:104664003031320033343500363738003961620076
:10467400636465006600300031323300343536003f
:1046840037383900414243004445460000000000e9
:044694000000000022
:020000040000fa
:104698000000fa0021e3a90021a3a9002143a800f2
:1046a8001132200091407800c0cfb30000c06000f4
:1046b80021e3b700013220009140780000ceb3001a
:1046c80000c0700020e3b7002043a9002023a90000
:1046d8002003a90023c3bf007f40600023e3b70085
:1046e8002223a9002203a90025e3a90025c3bf00ae
:1046f800f041b30025e3b700f0c3b30024e3b700eb
:104708000080eb00501988000080fa0000000600c5
:104718000400fa00000f780028e3a9001e40780082
:104728007f416000813220009140780000ceb300c4
:1047380000c060000240700028e3b7000000eb00f2
:1047480070198800110020001e0078000008dd00a4
:10475800801988000080eb005019880011002000a3
:104768001e0078000008dd000080ea00601988005b
:1047780021e3a8002023a80020c3bf000080fb007d
:10478800610060000000e000fbff320000188000bc
:10479800100798002023a90021e3a9001e0090001b
:0847a8000080fa000000060089
:020000040000fa
:1047b0000400fa00ca22a80000242400f10020000e
:1047c000008fbe001e00be00e00f5000e08f5800ba
:1047d000050035000080eb008080eb001e0f4000dc
:1047e0005e974800f7ff3700ca22a9000024240082
:1047f000f1002000008fbe001e00be00e00f500040
:10480000e08f5800050035000080eb008080eb0051
:104810001e0f40005e974800f7ff37000080fa0047
:10482000000006000400fa00caa2a8000024240028
:10483000f1002000008fbe001e00be00e00f5000ff
:10484000e08f5800050035000080eb008080eb0011
:104850001e0f40005e974800f7ff3700caa2a9006c
:1048600000242400f1002000008fbe001e00be00c6
:10487000e00f5000e08f5800050035000080eb008d
:104880008080eb001e0f40005e974800f7ff370066
:084890000080fa0000000600a0
:020000040000fa
:10489800809fbe008560a9004428ec00004280008b
:1048a800f003b20001802000810040000000eb000e
:1048b80026c2bf00804878004028ec004f00be00a8
:1048c80000400600004280001142800001005000b4
:1048d8000000060001428000124280000208e10048
:1048e80008003200f203b20001802000028140007b
:1048f80092407800014878004228ec00100020001f
:0c490800000006000000eb0000000600ac
:020000040000fa
:10491400809fbe0087c0a9008a28ec003044800034
:10492400f003b20061842000810040000000eb002d
:1049340036c2bf00804878008628ec004f00be00d5
:1049440000400600304480004144800001005000d3
:104954000000060031448000424480000208e10067
:1049640008003200f203b20061842000028140009a
:1049740092407800014878008828ec00100020005c
:0c498400000006000000eb000000060030
:020000040000fa
:104990000000fa00ca22a900c622a900caa2a900e2
:1049a000c6a2a900e4c2a900e4e2a800e502a900a9
:1049b000e522a900d302a900c602a800cb22a900c3
:1049c000c722a900d362a8000080fa0000000600f8
:020000040000fa
:1049d000f03fb1000180b10006003500ee03090090
:1049e00000000000403fb1000180b100fbff3d002e
:1049f0001000b000203fb000020035000080090028
:084a00000000000000000600a8
:020000040000fa
:044a08000000fe00ac
:00000001FF
